
 DRWATSON

 Start     Length     Name                   Class
 0001:0000 04062H     _TEXT                  CODE
 0002:0000 00001H     FAR_BSS                FAR_BSS
 0003:0000 00010H     NULL                   BEGDATA
 0003:0010 00C58H     _DATA                  DATA
 0003:0C68 0000EH     CDATA                  DATA
 0003:0C76 00000H     XIFB                   DATA
 0003:0C76 00000H     XIF                    DATA
 0003:0C76 00000H     XIFE                   DATA
 0003:0C76 00000H     XIB                    DATA
 0003:0C76 00000H     XI                     DATA
 0003:0C76 00000H     XIE                    DATA
 0003:0C76 00000H     XPB                    DATA
 0003:0C76 00000H     XP                     DATA
 0003:0C76 00000H     XPE                    DATA
 0003:0C76 00000H     XCB                    DATA
 0003:0C76 00000H     XC                     DATA
 0003:0C76 00000H     XCE                    DATA
 0003:0C76 00000H     XCFB                   DATA
 0003:0C76 00000H     XCF                    DATA
 0003:0C76 00000H     XCFE                   DATA
 0003:0C76 0000CH     DBDATA                 DATA
 0003:0C82 00002H     XIQC                   DATA
 0003:0C84 00000H     CONST                  CONST
 0003:0C84 00019H     HDR                    MSG
 0003:0C9D 000B1H     MSG                    MSG
 0003:0D4E 00002H     PAD                    MSG
 0003:0D50 00001H     EPAD                   MSG
 0003:0D60 001E0H     _BSS                   BSS
 0003:0F40 00000H     XOB                    BSS
 0003:0F40 00000H     XO                     BSS
 0003:0F40 00000H     XOE                    BSS
 0003:0F40 00436H     c_common               BSS

 Origin   Group
 0003:0   DGROUP

 Address   Export                  Alias

 0001:086A SherlockDialog          SherlockDialog
 0001:1A88 SherlockWndProc         SherlockWndProc

  Address         Publics by Name

 0000:0000  Imp  CLOSESOUND           (SOUND.2)
 0000:0000  Imp  CREATEWINDOW         (USER.41)
 0000:0000  Imp  DEFWINDOWPROC        (USER.107)
 0000:0000  Imp  DESTROYWINDOW        (USER.53)
 0000:0000  Imp  DIALOGBOX            (USER.87)
 0000:0000  Imp  DISPATCHMESSAGE      (USER.114)
 0000:0000  Imp  DOS3CALL             (KERNEL.102)
 0000:0000  Imp  ENDDIALOG            (USER.88)
 0000:0000  Imp  FATALAPPEXIT         (KERNEL.137)
 0000:0000  Imp  FATALEXIT            (KERNEL.1)
 0000:0000  Imp  FREEPROCINSTANCE     (KERNEL.52)
 0000:0000  Imp  GETCURRENTTASK       (KERNEL.36)
 0000:0000  Imp  GETDLGITEM           (USER.91)
 0000:0000  Imp  GETFREESPACE         (KERNEL.169)
 0000:0000  Imp  GETMESSAGE           (USER.108)
 0000:0000  Imp  GETMODULEHANDLE      (KERNEL.47)
 0000:0000  Imp  GETNUMTASKS          (KERNEL.152)
 0000:0000  Imp  GETPROFILEINT        (KERNEL.57)
 0000:0000  Imp  GETPROFILESTRING     (KERNEL.58)
 0000:0000  Imp  GETSTOCKOBJECT       (GDI.87)
 0000:0000  Imp  GETSYSTEMMETRICS     (USER.179)
 0000:0000  Imp  GETVERSION           (KERNEL.3)
 0000:0000  Imp  GETWINDOWSDIRECTORY  (KERNEL.134)
 0000:0000  Imp  GETWINFLAGS          (KERNEL.132)
 0000:0000  Imp  GLOBALALLOC          (KERNEL.15)
 0000:0000  Imp  GLOBALENTRYHANDLE    (TOOLHELP.54)
 0000:0000  Imp  GLOBALFREE           (KERNEL.17)
 0000:0000  Imp  GLOBALLOCK           (KERNEL.18)
 0000:0000  Imp  GLOBALREALLOC        (KERNEL.16)
 0001:3558       GPFAULT
 0000:0000  Imp  INITAPP              (USER.5)
 0000:0000  Imp  INITTASK             (KERNEL.91)
 0000:0000  Imp  INTERRUPTREGISTER    (TOOLHELP.75)
 0000:0000  Imp  INTERRUPTUNREGISTER  (TOOLHELP.76)
 0000:0000  Imp  LOADCURSOR           (USER.173)
 0000:0000  Imp  LOADICON             (USER.174)
 0000:0000  Imp  LOADSTRING           (USER.176)
 0000:0000  Imp  LOCALALLOC           (KERNEL.5)
 0000:0000  Imp  LOCALFREE            (KERNEL.7)
 0000:0000  Imp  LOCALREALLOC         (KERNEL.6)
 0000:0000  Imp  LOCKSEGMENT          (KERNEL.23)
 0000:0000  Imp  LSTRCAT              (KERNEL.89)
 0000:0000  Imp  LSTRCMP              (USER.430)
 0000:0000  Imp  LSTRCPY              (KERNEL.88)
 0000:0000  Imp  MAKEPROCINSTANCE     (KERNEL.51)
 0000:0000  Imp  MEMMANINFO           (TOOLHELP.72)
 0000:0000  Imp  MESSAGEBOX           (USER.1)
 0000:0000  Imp  MODULEFINDHANDLE     (TOOLHELP.62)
 0000:0000  Imp  MODULEFINDNAME       (TOOLHELP.61)
 0000:0000  Imp  MODULEFIRST          (TOOLHELP.59)
 0000:0000  Imp  MODULENEXT           (TOOLHELP.60)
 0000:0000  Imp  NOTIFYREGISTER       (TOOLHELP.73)
 0000:0000  Imp  NOTIFYUNREGISTER     (TOOLHELP.74)
 0000:0000  Imp  OPENSOUND            (SOUND.1)
 0000:0000  Imp  OUTPUTDEBUGSTRING    (KERNEL.115)
 0000:0008  Abs  pAtomTable
 0000:0006  Abs  pLocalHeap
 0000:0000  Imp  POSTMESSAGE          (USER.110)
 0000:0000  Imp  POSTQUITMESSAGE      (USER.6)
 0000:000E  Abs  pStackBot
 0000:000C  Abs  pStackMin
 0000:000A  Abs  pStackTop
 0000:0000  Imp  REGISTERCLASS        (USER.57)
 0003:0004       rsrvptrs
 0000:0000  Imp  SENDMESSAGE          (USER.111)
 0000:0000  Imp  SETVOICESOUND        (SOUND.8)
 0001:086A       SherlockDialog
 0001:1A88       SherlockWndProc
 0000:0000  Imp  SHOWWINDOW           (USER.42)
 0000:0000  Imp  STACKTRACECSIPFIRST  (TOOLHELP.67)
 0000:0000  Imp  STACKTRACENEXT       (TOOLHELP.68)
 0000:0000  Imp  STARTSOUND           (SOUND.9)
 0003:0BF0       STKHQQ
 0000:0000  Imp  STOPSOUND            (SOUND.10)
 0000:0000  Imp  SYSERRORBOX          (USER.320)
 0000:0000  Imp  SYSTEMHEAPINFO       (TOOLHELP.71)
 0000:0000  Imp  TASKFINDHANDLE       (TOOLHELP.65)
 0000:0000  Imp  TASKFIRST            (TOOLHELP.63)
 0000:0000  Imp  TASKNEXT             (TOOLHELP.64)
 0000:0000  Imp  TERMINATEAPP         (TOOLHELP.77)
 0000:0000  Imp  TRANSLATEMESSAGE     (USER.113)
 0000:0000  Imp  UNLOCKSEGMENT        (KERNEL.24)
 0000:0000  Imp  UPDATEWINDOW         (USER.124)
 0000:0000  Imp  WAITEVENT            (KERNEL.30)
 0001:1BC2       WINMAIN
 0000:0000  Imp  WVSPRINTF            (USER.421)
 0003:1366       _adrSize
 0003:0FE8       _aszStrings
 0001:0E5A       _BeginReport
 0001:1E06       _BMid
 0003:136A       _bogus
 0001:1DE4       _BReg
 0003:03C4       _bregs
 0003:0F48       _bugCnt
 0001:34FC       _CallMe
 0001:1586       _CallMeToo
 0001:2386       _Cat0
 0001:2394       _Cat1
 0001:23B2       _Cat2
 0001:23D4       _Cat3
 0003:1312       _code
 0003:11FA       _cpu32
 0001:03BA       _CurModuleName
 0001:0458       _CurTime
 0003:0FE6       _dataSize
 0003:0FE0       _ddFlag
 0001:0188       _DecodeFault
 0003:00A6       _deltaPitch
 0001:32EE       _DisAsm386
 0001:2A08       _DisAsm86
 0001:060E       _DisAsmAround
 0001:23FA       _DisAsmF
 0003:009C       _disLen
 0003:00A2       _disStack
 0001:1E60       _DMid
 0001:1E3C       _DReg
 0003:03F4       _dregs
 0003:0972       _dsimple
 0001:09BC       _DumpInfo
 0001:0CC4       _DumpStack
 0001:3998       _dup
 0001:39F0       _dup2
 0003:0D60       _edata
 0003:1376       _end
 0001:0ED8       _EndReport
 0003:0C3F       _environ
 0003:0C18       _errno
 0001:3B49       _exit
 0001:02B4       _FaultCause
 0003:00A4       _fh
 0001:03F4       _FileInfo
 0001:36EC       _FindFile
 0001:3308       _FindSym
 0003:008C       _flBit
 0002:0000       _foo
 0001:1ED4       _GetByte
 0001:1F4C       _GetDWord
 0001:2010       _GetImmAdr
 0001:1F8E       _GetImmByte
 0001:2030       _GetImmData
 0001:1FF2       _GetImmDWord
 0001:1FD6       _GetImmWord
 0001:0C14       _GetProcName
 0001:3691       _GETREGS32
 0001:1FAC       _GetSImmByte
 0001:36C9       _GetTimeDate
 0001:1F14       _GetWord
 0003:0FB0       _gpRegs
 0003:0FDA       _gpSafe
 0003:0F40       _gpStack
 0003:042C       _grp1
 0003:044C       _grp2
 0003:046C       _grp3
 0003:0494       _grp5
 0003:04C4       _grp6
 0003:04EC       _grp7
 0003:0524       _grp8
 0003:0F5A       _hexData
 0003:0FDC       _hexPos
 0003:130E       _hInst
 0003:12FC       _hTask
 0003:11F6       _hWnd
 0003:00A0       _iFeelLucky
 0003:0F50       _immData
 0003:1310       _imTrying
 0003:0F42       _init
 0001:1D36       _InitDisAsm86
 0001:1A10       _InitSherlock
 0001:2954       _IsPrefix
 0003:057C       _jcond
 0001:2050       _JRel
 0003:12FE       _lastErr
 0000:0000  Imp  _LCLOSE              (KERNEL.81)
 0000:0000  Imp  _LCREAT              (KERNEL.83)
 0003:1370       _level
 0003:11A2       _line
 0000:0000  Imp  _LLSEEK              (KERNEL.84)
 0001:17CA       _LoadStringResources
 0001:3722       _LogErrorStr
 0003:1316       _logFile
 0001:3752       _LogParamErrorStr
 0003:11FC       _lookup
 0000:0000  Imp  _LOPEN               (KERNEL.85)
 0000:0000  Imp  _LREAD               (KERNEL.82)
 0000:0000  Imp  _LWRITE              (KERNEL.86)
 0001:3F4A       _malloc
 0003:0F84       _memDisp
 0003:136E       _memDouble
 0003:11F2       _memLinear
 0003:0F4A       _memLinear2
 0003:09F8       _memName
 0003:1372       _memOp
 0003:0F4E       _memOp2
 0003:0FB2       _memReg
 0003:0FD8       _memSeg
 0003:0FE4       _memSeg2
 0003:0F46       _memSize
 0003:0F82       _memSize2
 0001:2372       _ModRM
 0001:20C6       _ModRMGeneral
 0001:235E       _ModRMInfo
 0001:0126       _ModuleName
 0001:1A4E       _Moriarty
 0001:081C       _MyClose
 0001:05B0       _MyFlush
 0001:07C2       _MyOpen
 0001:343E       _NearestSym
 0003:1374       _newsp
 0003:06B2       _ops
 0001:172A       _ParseInfo
 0003:11F8       _pending
 0003:130A       _pitch
 0001:0940       _PrepareToParty
 0003:03C2       _preSeg
 0001:083E       _PutDate
 0001:1882       _ReadWinIni
 0003:0FB6       _regs
 0003:0F88       _regs32
 0003:11A0       _retflag
 0003:0A48       _rms
 0001:0276       _SafeDisAsm86
 0001:34D0       _SegBase
 0001:0010       _SegFlags
 0001:00BA       _SegInfo
 0001:349E       _SegLimit
 0001:00F6       _SegNum
 0001:34ED       _SegRights
 0003:0F44       _segSize
 0001:0F92       _Sherlock
 0001:0526       _Show
 0001:0F38       _ShowParamError
 0003:0896       _simple
 0003:1368       _sound
 0003:0414       _sregs
 0001:38D0       _strcat
 0001:3A28       _strchr
 0001:3910       _strcpy
 0003:09C2       _stringOp
 0001:3942       _strlen
 0001:3A52       _strlwr
 0001:395E       _strncmp
 0003:0046       _syms
 0003:0010       _szAppName
 0003:001C       _szAppNameShort
 0003:0026       _szAppNameShortLog
 0001:04B0       _Tab2Spc
 0003:009E       _trapZero
 0001:1E90       _VMid
 0001:1E74       _VReg
 0003:00AA       _wf
 0003:0FDE       _whined
 0001:1E1A       _WReg
 0003:03DC       _wregs
 0000:0000  Imp  _wsprintf            (USER.420)
 0001:1EBE       _XMid
 0001:1EA4       _XReg
 0003:0BFC       __acfinfo
 0000:9876  Abs  __acrtmsg
 0000:9876  Abs  __acrtused
 0000:9876  Abs  __acrtused2
 0000:D6D6  Abs  __aDBdoswp
 0003:0C4E       __adbgmsg
 0003:0C7A       __aDBrterr
 0003:0C0A       __aintdiv
 0003:0C66       __amblksiz
 0001:3EAF       __amsg_exit
 0001:3A70       __aNlshl
 0001:3863       __astart
 0003:0C8C       __caption
 0001:3B58       __cexit
 0003:0C46       __child
 0001:3A7C       __cinit
 0001:3EAA       __cintDIV
 0001:3BC2       __ctermsub
 0001:3B62       __c_exit
 0003:0C23       __doserrno
 0001:3E4E       __dosret0
 0001:3E63       __dosretax
 0001:3E56       __dosreturn
 0003:0C20       __dosvermajor
 0003:0C21       __dosverminor
 0003:0D60       __edata
 0003:1376       __end
 0001:3B50       __exit
 0003:0C0E       __fac
 0001:3FC2       __ffree
 0001:3F98       __fmalloc
 0003:0C6A       __fpinit
 0000:9876  Abs  __fptaskdata
 0001:3EA4       __fptrap
 0001:4022       __frealloc
 0003:0C49       __intno
 0001:3E70       __maperror
 0001:3F1E       __myalloc
 0003:0C25       __nfile
 0001:3F88       __nfree
 0001:3F4E       __nmalloc
 0001:3ECC       __NMSG_TEXT
 0001:3EF7       __NMSG_WRITE
 0001:3FD2       __nrealloc
 0003:0C23       __oserr
 0003:0C27       __osfile
 0003:0C20       __osmajor
 0003:0C21       __osminor
 0003:0C22       __osmode
 0003:0C20       __osversion
 0003:0C48       __ovlflag
 0003:0C4A       __ovlvec
 0003:0C41       __pgmptr
 0003:0C1E       __psp
 0003:0C1C       __pspadr
 0001:3C32       __setargv
 0001:3DD0       __setenvp
 0003:0C1A       __umaskval
 0001:3861       __wflags
 0000:0000  Imp  __WINFLAGS           (KERNEL.178)
 0003:0C7C       ___aDBexit
 0003:0C78       ___aDBswpchk
 0003:0C76       ___aDBswpflg
 0003:0C3B       ___argc
 0003:0C3D       ___argv
 0003:0C82       ___qczrinit

  Address         Publics by Value

 0000:0000  Imp  _LWRITE              (KERNEL.86)
 0000:0000  Imp  STACKTRACECSIPFIRST  (TOOLHELP.67)
 0000:0000  Imp  STARTSOUND           (SOUND.9)
 0000:0000  Imp  GETVERSION           (KERNEL.3)
 0000:0000  Imp  GLOBALFREE           (KERNEL.17)
 0000:0000  Imp  UPDATEWINDOW         (USER.124)
 0000:0000  Imp  INITTASK             (KERNEL.91)
 0000:0000  Imp  GLOBALENTRYHANDLE    (TOOLHELP.54)
 0000:0000  Imp  _LCREAT              (KERNEL.83)
 0000:0000  Imp  FATALEXIT            (KERNEL.1)
 0000:0000  Imp  SHOWWINDOW           (USER.42)
 0000:0000  Imp  DISPATCHMESSAGE      (USER.114)
 0000:0000  Imp  MODULEFINDNAME       (TOOLHELP.61)
 0000:0000  Imp  DOS3CALL             (KERNEL.102)
 0000:0000  Imp  FREEPROCINSTANCE     (KERNEL.52)
 0000:0000  Imp  POSTMESSAGE          (USER.110)
 0000:0000  Imp  GLOBALREALLOC        (KERNEL.16)
 0000:0000  Imp  MESSAGEBOX           (USER.1)
 0000:0000  Imp  __WINFLAGS           (KERNEL.178)
 0000:0000  Imp  GETPROFILESTRING     (KERNEL.58)
 0000:0000  Imp  GETWINFLAGS          (KERNEL.132)
 0000:0000  Imp  GLOBALALLOC          (KERNEL.15)
 0000:0000  Imp  WVSPRINTF            (USER.421)
 0000:0000  Imp  LSTRCPY              (KERNEL.88)
 0000:0000  Imp  GETMODULEHANDLE      (KERNEL.47)
 0000:0000  Imp  LSTRCAT              (KERNEL.89)
 0000:0000  Imp  TASKNEXT             (TOOLHELP.64)
 0000:0000  Imp  DEFWINDOWPROC        (USER.107)
 0000:0000  Imp  INTERRUPTUNREGISTER  (TOOLHELP.76)
 0000:0000  Imp  POSTQUITMESSAGE      (USER.6)
 0000:0000  Imp  STOPSOUND            (SOUND.10)
 0000:0000  Imp  LOADCURSOR           (USER.173)
 0000:0000  Imp  TERMINATEAPP         (TOOLHELP.77)
 0000:0000  Imp  GETSYSTEMMETRICS     (USER.179)
 0000:0000  Imp  SENDMESSAGE          (USER.111)
 0000:0000  Imp  LSTRCMP              (USER.430)
 0000:0000  Imp  GETSTOCKOBJECT       (GDI.87)
 0000:0000  Imp  LOCKSEGMENT          (KERNEL.23)
 0000:0000  Imp  INITAPP              (USER.5)
 0000:0000  Imp  TRANSLATEMESSAGE     (USER.113)
 0000:0000  Imp  REGISTERCLASS        (USER.57)
 0000:0000  Imp  LOCALALLOC           (KERNEL.5)
 0000:0000  Imp  GETFREESPACE         (KERNEL.169)
 0000:0000  Imp  TASKFIRST            (TOOLHELP.63)
 0000:0000  Imp  _LOPEN               (KERNEL.85)
 0000:0000  Imp  OPENSOUND            (SOUND.1)
 0000:0000  Imp  LOADICON             (USER.174)
 0000:0000  Imp  SYSERRORBOX          (USER.320)
 0000:0000  Imp  LOADSTRING           (USER.176)
 0000:0000  Imp  _LCLOSE              (KERNEL.81)
 0000:0000  Imp  MAKEPROCINSTANCE     (KERNEL.51)
 0000:0000  Imp  TASKFINDHANDLE       (TOOLHELP.65)
 0000:0000  Imp  INTERRUPTREGISTER    (TOOLHELP.75)
 0000:0000  Imp  DIALOGBOX            (USER.87)
 0000:0000  Imp  MODULEFINDHANDLE     (TOOLHELP.62)
 0000:0000  Imp  GETPROFILEINT        (KERNEL.57)
 0000:0000  Imp  NOTIFYUNREGISTER     (TOOLHELP.74)
 0000:0000  Imp  GETDLGITEM           (USER.91)
 0000:0000  Imp  GLOBALLOCK           (KERNEL.18)
 0000:0000  Imp  DESTROYWINDOW        (USER.53)
 0000:0000  Imp  GETCURRENTTASK       (KERNEL.36)
 0000:0000  Imp  STACKTRACENEXT       (TOOLHELP.68)
 0000:0000  Imp  CREATEWINDOW         (USER.41)
 0000:0000  Imp  CLOSESOUND           (SOUND.2)
 0000:0000  Imp  _wsprintf            (USER.420)
 0000:0000  Imp  ENDDIALOG            (USER.88)
 0000:0000  Imp  NOTIFYREGISTER       (TOOLHELP.73)
 0000:0000  Imp  LOCALREALLOC         (KERNEL.6)
 0000:0000  Imp  WAITEVENT            (KERNEL.30)
 0000:0000  Imp  MEMMANINFO           (TOOLHELP.72)
 0000:0000  Imp  UNLOCKSEGMENT        (KERNEL.24)
 0000:0000  Imp  MODULEFIRST          (TOOLHELP.59)
 0000:0000  Imp  GETMESSAGE           (USER.108)
 0000:0000  Imp  _LREAD               (KERNEL.82)
 0000:0000  Imp  FATALAPPEXIT         (KERNEL.137)
 0000:0000  Imp  SETVOICESOUND        (SOUND.8)
 0000:0000  Imp  MODULENEXT           (TOOLHELP.60)
 0000:0000  Imp  GETWINDOWSDIRECTORY  (KERNEL.134)
 0000:0000  Imp  SYSTEMHEAPINFO       (TOOLHELP.71)
 0000:0000  Imp  _LLSEEK              (KERNEL.84)
 0000:0000  Imp  GETNUMTASKS          (KERNEL.152)
 0000:0000  Imp  OUTPUTDEBUGSTRING    (KERNEL.115)
 0000:0000  Imp  LOCALFREE            (KERNEL.7)
 0000:0006  Abs  pLocalHeap
 0000:0008  Abs  pAtomTable
 0000:000A  Abs  pStackTop
 0000:000C  Abs  pStackMin
 0000:000E  Abs  pStackBot
 0000:9876  Abs  __acrtmsg
 0000:9876  Abs  __acrtused
 0000:9876  Abs  __acrtused2
 0000:9876  Abs  __fptaskdata
 0000:D6D6  Abs  __aDBdoswp
 0001:0010       _SegFlags
 0001:00BA       _SegInfo
 0001:00F6       _SegNum
 0001:0126       _ModuleName
 0001:0188       _DecodeFault
 0001:0276       _SafeDisAsm86
 0001:02B4       _FaultCause
 0001:03BA       _CurModuleName
 0001:03F4       _FileInfo
 0001:0458       _CurTime
 0001:04B0       _Tab2Spc
 0001:0526       _Show
 0001:05B0       _MyFlush
 0001:060E       _DisAsmAround
 0001:07C2       _MyOpen
 0001:081C       _MyClose
 0001:083E       _PutDate
 0001:086A       SherlockDialog
 0001:0940       _PrepareToParty
 0001:09BC       _DumpInfo
 0001:0C14       _GetProcName
 0001:0CC4       _DumpStack
 0001:0E5A       _BeginReport
 0001:0ED8       _EndReport
 0001:0F38       _ShowParamError
 0001:0F92       _Sherlock
 0001:1586       _CallMeToo
 0001:172A       _ParseInfo
 0001:17CA       _LoadStringResources
 0001:1882       _ReadWinIni
 0001:1A10       _InitSherlock
 0001:1A4E       _Moriarty
 0001:1A88       SherlockWndProc
 0001:1BC2       WINMAIN
 0001:1D36       _InitDisAsm86
 0001:1DE4       _BReg
 0001:1E06       _BMid
 0001:1E1A       _WReg
 0001:1E3C       _DReg
 0001:1E60       _DMid
 0001:1E74       _VReg
 0001:1E90       _VMid
 0001:1EA4       _XReg
 0001:1EBE       _XMid
 0001:1ED4       _GetByte
 0001:1F14       _GetWord
 0001:1F4C       _GetDWord
 0001:1F8E       _GetImmByte
 0001:1FAC       _GetSImmByte
 0001:1FD6       _GetImmWord
 0001:1FF2       _GetImmDWord
 0001:2010       _GetImmAdr
 0001:2030       _GetImmData
 0001:2050       _JRel
 0001:20C6       _ModRMGeneral
 0001:235E       _ModRMInfo
 0001:2372       _ModRM
 0001:2386       _Cat0
 0001:2394       _Cat1
 0001:23B2       _Cat2
 0001:23D4       _Cat3
 0001:23FA       _DisAsmF
 0001:2954       _IsPrefix
 0001:2A08       _DisAsm86
 0001:32EE       _DisAsm386
 0001:3308       _FindSym
 0001:343E       _NearestSym
 0001:349E       _SegLimit
 0001:34D0       _SegBase
 0001:34ED       _SegRights
 0001:34FC       _CallMe
 0001:3558       GPFAULT
 0001:3691       _GETREGS32
 0001:36C9       _GetTimeDate
 0001:36EC       _FindFile
 0001:3722       _LogErrorStr
 0001:3752       _LogParamErrorStr
 0001:3861       __wflags
 0001:3863       __astart
 0001:38D0       _strcat
 0001:3910       _strcpy
 0001:3942       _strlen
 0001:395E       _strncmp
 0001:3998       _dup
 0001:39F0       _dup2
 0001:3A28       _strchr
 0001:3A52       _strlwr
 0001:3A70       __aNlshl
 0001:3A7C       __cinit
 0001:3B49       _exit
 0001:3B50       __exit
 0001:3B58       __cexit
 0001:3B62       __c_exit
 0001:3BC2       __ctermsub
 0001:3C32       __setargv
 0001:3DD0       __setenvp
 0001:3E4E       __dosret0
 0001:3E56       __dosreturn
 0001:3E63       __dosretax
 0001:3E70       __maperror
 0001:3EA4       __fptrap
 0001:3EAA       __cintDIV
 0001:3EAF       __amsg_exit
 0001:3ECC       __NMSG_TEXT
 0001:3EF7       __NMSG_WRITE
 0001:3F1E       __myalloc
 0001:3F4A       _malloc
 0001:3F4E       __nmalloc
 0001:3F88       __nfree
 0001:3F98       __fmalloc
 0001:3FC2       __ffree
 0001:3FD2       __nrealloc
 0001:4022       __frealloc
 0002:0000       _foo
 0003:0004       rsrvptrs
 0003:0010       _szAppName
 0003:001C       _szAppNameShort
 0003:0026       _szAppNameShortLog
 0003:0046       _syms
 0003:008C       _flBit
 0003:009C       _disLen
 0003:009E       _trapZero
 0003:00A0       _iFeelLucky
 0003:00A2       _disStack
 0003:00A4       _fh
 0003:00A6       _deltaPitch
 0003:00AA       _wf
 0003:03C2       _preSeg
 0003:03C4       _bregs
 0003:03DC       _wregs
 0003:03F4       _dregs
 0003:0414       _sregs
 0003:042C       _grp1
 0003:044C       _grp2
 0003:046C       _grp3
 0003:0494       _grp5
 0003:04C4       _grp6
 0003:04EC       _grp7
 0003:0524       _grp8
 0003:057C       _jcond
 0003:06B2       _ops
 0003:0896       _simple
 0003:0972       _dsimple
 0003:09C2       _stringOp
 0003:09F8       _memName
 0003:0A48       _rms
 0003:0BF0       STKHQQ
 0003:0BFC       __acfinfo
 0003:0C0A       __aintdiv
 0003:0C0E       __fac
 0003:0C18       _errno
 0003:0C1A       __umaskval
 0003:0C1C       __pspadr
 0003:0C1E       __psp
 0003:0C20       __dosvermajor
 0003:0C20       __osmajor
 0003:0C20       __osversion
 0003:0C21       __osminor
 0003:0C21       __dosverminor
 0003:0C22       __osmode
 0003:0C23       __doserrno
 0003:0C23       __oserr
 0003:0C25       __nfile
 0003:0C27       __osfile
 0003:0C3B       ___argc
 0003:0C3D       ___argv
 0003:0C3F       _environ
 0003:0C41       __pgmptr
 0003:0C46       __child
 0003:0C48       __ovlflag
 0003:0C49       __intno
 0003:0C4A       __ovlvec
 0003:0C4E       __adbgmsg
 0003:0C66       __amblksiz
 0003:0C6A       __fpinit
 0003:0C76       ___aDBswpflg
 0003:0C78       ___aDBswpchk
 0003:0C7A       __aDBrterr
 0003:0C7C       ___aDBexit
 0003:0C82       ___qczrinit
 0003:0C8C       __caption
 0003:0D60       _edata
 0003:0D60       __edata
 0003:0F40       _gpStack
 0003:0F42       _init
 0003:0F44       _segSize
 0003:0F46       _memSize
 0003:0F48       _bugCnt
 0003:0F4A       _memLinear2
 0003:0F4E       _memOp2
 0003:0F50       _immData
 0003:0F5A       _hexData
 0003:0F82       _memSize2
 0003:0F84       _memDisp
 0003:0F88       _regs32
 0003:0FB0       _gpRegs
 0003:0FB2       _memReg
 0003:0FB6       _regs
 0003:0FD8       _memSeg
 0003:0FDA       _gpSafe
 0003:0FDC       _hexPos
 0003:0FDE       _whined
 0003:0FE0       _ddFlag
 0003:0FE4       _memSeg2
 0003:0FE6       _dataSize
 0003:0FE8       _aszStrings
 0003:11A0       _retflag
 0003:11A2       _line
 0003:11F2       _memLinear
 0003:11F6       _hWnd
 0003:11F8       _pending
 0003:11FA       _cpu32
 0003:11FC       _lookup
 0003:12FC       _hTask
 0003:12FE       _lastErr
 0003:130A       _pitch
 0003:130E       _hInst
 0003:1310       _imTrying
 0003:1312       _code
 0003:1316       _logFile
 0003:1366       _adrSize
 0003:1368       _sound
 0003:136A       _bogus
 0003:136E       _memDouble
 0003:1370       _level
 0003:1372       _memOp
 0003:1374       _newsp
 0003:1376       _end
 0003:1376       __end

Program entry point at 0001:3863
